:020000040000FA
:0400000005303A2865
:08000800A000030EA100831209
:1000100005191028831601178312B23081002B288E
:1000200083160113831203140B190310A80DA90DD5
:10003000AA0DAB0DAC0DAC16FF302C02031D2B2806
:10004000FA302B02031D2B2831152A08AF0029088E
:10005000AE002808AD008B100B11210E8300A00EFE
:04006000200E090065
:0C007400203084008001840A6030040207
:10008000031C3C281230B00088218316FF23900007
:10009000831283160C308505870183128501870141
:1000A000073099000030831691009F008312C830FA
:1000B00083168100831231309000003083168C004B
:1000C000831210308B00C62181018E018F010B112C
:1000D0008B100B108C018B177B2031197E20B30BFA
:1000E0007928031085190314B90DF030390203196A
:1000F0000321D3216C286400321008003111013033
:10010000B7008B132030370783169B001C141A0886
:100110008312A4001030370783169B001C141A08A2
:100120008312A300A6000230A6060030370783160C
:100130009B001C141A088312A200A7000130A70616
:100140008B17321CA92822090339A200A309A4098C
:10015000A50924082F02031DFD2823082E02031DD4
:10016000FD2822082D02031DFD2801303702031D42
:10017000BE283D18BE283D143E1496210230370299
:10018000031DC728BD18C728BD143E149C21033089
:100190003702031DD0283D19D0283D153E14A22159
:1001A00004303702031DD928BD19D928BD153E14C6
:1001B000A82105303702031DE2283D1AE2283D162A
:1001C0003E14AE2106303702031DEB28BD1AEB2882
:1001D000BD163E14AF2107303702031DF4283D1B26
:1001E000F4283D173E14B02108303702031DFD28C6
:1001F000BD1BFD28BD173E14B121B70A05303702DB
:100200000318080081280130B600B300B400B5001F
:10021000B70085018701B1137B20B30B3B29031085
:1002200085190314B90DF030390203196229B40B92
:100230003B29013037020319B2210230370203197A
:10024000B621033037020319BA21043037020319EB
:10025000BE21053037020319C221063037020319C7
:10026000C321073037020319C421083037020319AC
:10027000C5219630B400311D0C293111321C45299D
:100280002D090339AD00AE09AF092F1C0C298E01D1
:100290008F010C1C0C290C102E1E0C298B132030E6
:1002A0003707BB002F08BA00752110303707BB0095
:1002B0002E08BA00752100303707BB002D08BA00A0
:1002C00075218B1785018701B70AB6010530370202
:1002D000031C0C29C62108003E1C08003E101030EB
:1002E000BB003D08BA00752108008B133A0883163D
:1002F0001C159A003B089B0055309D00AA309D00BC
:100300009C1464009C1881291C1183128B1708000F
:10031000831610309B001C141A088312BD00FF3096
:10032000D000D415D515D615D71508000F30D20436
:10033000BD103D11BD1108000F30D2043D103D111C
:10034000BD1108000F30D2043D10BD10BD110800D2
:100350000F30D2043D10BD103D1108000800080008
:10036000080008000508023A850008000508013A5F
:10037000850008000508203A850008000508103AA5
:100380008500080008000800080008006400B30B9E
:10039000C629B40BC6293D08D200031D0800113040
:1003A000BD00D20008008F08031908008F01D00F8C
:1003B000612AD00A0E305205031DED29541DE32990
:1003C000D4015416FB29D41DE829D4015416FB2965
:1003D000541EFB29D401D414FB29D41CF229D401C6
:1003E0005415FB29541DF729D401D415FB29541E9B
:1003F000FB29D40154150D305205031D0E2A551D3D
:10040000042AD50155161C2AD51D092AD5015516D1
:100410001C2A551E1C2AD501D5141C2AD51C132AAA
:10042000D50155151C2A551D182AD501D5151C2A8C
:10043000551E1C2AD50155150B305205031D2F2AB8
:10044000561D252AD60156163D2AD61D2A2AD60122
:1004500056163D2A561E3D2AD601D6143D2AD61CD4
:10046000342AD60156153D2A561D392AD601D615ED
:100470003D2A561E3D2AD601561507305205031D4A
:10048000502A571D462AD70157165E2AD71D4B2AD8
:10049000D70157165E2A571E5E2AD701D7145E2A47
:1004A000D71C552AD70157155E2A571D5A2AD7013E
:1004B000D7155E2A571E5E2AD70157156C213D08B5
:1004C000D2005008D1000C305405031D85100C30AB
:1004D0005505031D05100C305605031D85120C3003
:1004E0005705031D051251080E0203188B2A1230FE
:1004F0005405031D851412305505031D05141230D3
:100500005605031D851612305705031D0516FF30CD
:100510005002031908008F08031D08007B205108B2
:100520000E02031C8B2A18305405031D851006305B
:100530005405031D851418305505031D051006309C
:100540005505031D051418305605031D8512063088
:100550005605031D851618305705031D0512063074
:080560005705031D05160800F4
:084000000400030006000400A7
:02400E00CC01E3
:10420000010078007A007C007E007B0079007F004E
:104210007D007A0078007E007C00FF00FF00FF0038
:104220000000F200F600FA00FE00F200F600FA00CC
:10423000FE00F200F600FA00FE00FF00FF00FF00A3
:10424000010005000500050005000900090009003E
:1042500009000D000D000D000D00FF00FF00FF0024
:10426000FF00FF00FF00FF00FF00FF00FF00FF0056
:10427000FF00FF00FF00FF00FF00FF00FF00FF0046
:10428000FF00FF00FF00FF00FF00FF00FF00FF0036
:10429000FF00FF00FF00FF00FF00FF00FF00FF0026
:1042A000FF00FF00FF00FF00FF00FF00FF00FF0016
:1042B000FF00FF00FF00FF00FF00FF00FF00FF0006
:1042C000FF00FF00FF00FF00FF00FF00FF00FF00F6
:1042D000FF00FF00FF00FF00FF00FF00FF00FF00E6
:1042E000FF00FF00FF00FF00FF00FF00FF00FF00D6
:1042F000FF00FF00FF00FF00FF00FF00FF00DD00E8
:00000001FF
